:020000023000CC
:10E000000D94B9F20D94E2F20D94E2F20D94E2F265
:10E010000D94E2F20D94E2F20D94E2F20D94E2F22C
:10E020000D94E2F20D94E2F20D94E2F20D94E2F21C
:10E030000D94E2F20D94E2F20D94E2F20D94E2F20C
:10E040000D94E2F20D94E2F20D94E2F20D94E2F2FC
:10E050000D94E2F20D94E2F20D94E2F20D94E2F2EC
:10E060000D94E2F20D94E2F20D94E2F20D94E2F2DC
:10E070000D94E2F20D94E2F20D94E2F20D94E2F2CC
:10E080000D94E2F20D94E2F20D94E2F20D94E2F2BC
:10E090000D94E2F20D94E2F20D94E2F20D94E2F2AC
:10E0A0000D94E2F20D94E2F20D94E2F20D94E2F29C
:10E0B0000D94E2F20D94E2F20D94E2F20D94E2F28C
:10E0C0000D94E2F20D94E2F20D94E2F241546D658A
:10E0D0006761323536310041726475696E6F206553
:10E0E00078706C6F7265722073746B353030563295
:10E0F000206279204D4C5300426F6F746C6F6164E5
:10E1000065723E004875683F00436F6D70696C65CD
:10E1100064206F6E20203D200043505520547970BC
:10E120006520202020203D20005F5F4156525F4146
:10E130005243485F5F203D2000415652204C6962A7
:10E140004320566572203D200047434320566572A8
:10E1500073696F6E20203D2000435055207369671E
:10E160006E61747572653D20004C6F772066757323
:10E170006520202020203D200048696768206675C2
:10E180007365202020203D2000457874206675733B
:10E190006520202020203D20004C6F636B20667599
:10E1A0007365202020203D20004D617920333120EF
:10E1B0003230313100312E362E3700342E332E33AB
:10E1C000005623202020414444522020206F7020FC
:10E1D000636F64652020202020696E7374727563FC
:10E1E00074696F6E2061646472202020496E7465CA
:10E1F0007272757074006E6F20766563746F720052
:10E20000726A6D702020006A6D702000576861741A
:10E2100020706F72743A00506F7274206E6F7420A9
:10E22000737570706F72746564004D7573742062DD
:10E23000652061206C6574746572002000577269F6
:10E240007474696E672045450052656164696E6744
:10E2500020454500656570726F6D206572726F7242
:10E2600020636F756E743D00504F525400303D5A1C
:10E2700065726F2061646472657373206374727376
:10E28000003F3D43505520737461747300403D4519
:10E290004550524F4D207465737400423D426C6985
:10E2A0006E6B204C454400453D44756D70204545DE
:10E2B00050524F4D00463D44756D7020464C4153C1
:10E2C0004800483D48656C70004C3D4C69737420B3
:10E2D000492F4F20506F72747300513D517569740E
:10E2E0002026206A756D7020746F2075736572200A
:10E2F00070676D00523D44756D702052414D00565F
:10E300003D73686F7720696E7465727275707420E2
:10E31000566563746F727300593D506F727420625A
:10E320006C696E6B002A00524553455400494E54A7
:10E330003000494E543100494E543200494E543356
:10E3400000494E543400494E543500494E5436006D
:10E35000494E5437005043494E5430005043494EC3
:10E360005431005744540054494D45523020434FD6
:10E370004D50410054494D45523020434F4D50427D
:10E380000054494D455230204F56460054494D45A2
:10E39000523120434150540054494D45523120439D
:10E3A0004F4D50410054494D45523120434F4D503F
:10E3B000420054494D45523120434F4D5043005483
:10E3C000494D455231204F56460054494D45523231
:10E3D00020434F4D50410054494D45523220434F48
:10E3E0004D50420054494D455232204F564600543C
:10E3F000494D45523320434150540054494D4552F4
:10E400003320434F4D50410054494D455233204332
:10E410004F4D50420054494D45523320434F4D50CB
:10E42000430054494D455233204F56460054494D00
:10E4300045523420434F4D50410054494D455234CC
:10E4400020434F4D50420054494D45523420434FD4
:10E450004D50430054494D455234204F56460054C8
:10E46000494D45523520434F4D50410054494D458B
:10E47000523520434F4D50420054494D45523520AE
:10E48000434F4D50430054494D455235204F564659
:10E490000055534152543020525800555341525464
:10E4A0003020554452450055534152543020545861
:10E4B0000055534152543120525800555341525443
:10E4C000312055445245005553415254312054583F
:10E4D00000535049205354430041444300414E41AE
:10E4E0004C4F4720434F4D50004545205245414435
:10E4F00059005457490053504D205245414459004A
:10E500004E4F545F55534544002A0027E32DE33214
:10E51000E337E33CE341E346E34BE350E355E35C9D
:10E52000E300E563E3CAE3D7E3E4E38CE398E3A520
:10E53000E3B2E3BFE367E374E381E3D1E491E49BF7
:10E54000E4A7E4DDE4D9E4E9E4EFE3FBE308E41560
:10E55000E422E4B1E4BBE4C7E4F2E4F6E400E52D30
:10E56000E43AE447E454E400E55FE46CE479E486EB
:10E57000E40011241FBECFEFD1E2DEBFCDBF01E02A
:10E580000CBF12E0A0E0B2E0EAEFFDEF03E00BBF4A
:10E5900002C007900D92A030B107D9F712E0A0E0B9
:10E5A000B2E001C01D92AC30B107E1F70F94ACF4BA
:10E5B0000D94FBFE01E20EBF0FEF0DBF11241FBE35
:10E5C0000D94ACF40D9400F020E030E040ED57E005
:10E5D00005C0FA013197F1F72F5F3F4F2817390730
:10E5E000C0F308959C01442737FD4095542FDA016C
:10E5F000C901860F911DA11DB11DABBFFC01879103
:10E60000882369F08093CE008091C80086FFFCCFFC
:10E610008091C80080648093C8006F5FE8CF089540
:10E620008DE08093CE008091C80086FFFCCF809162
:10E63000C80080648093C8008AE08093CE008091F7
:10E64000C80086FFFCCF8091C80080648093C8001A
:10E6500008950F94F2F20F9410F30895FC01908145
:10E66000992359F09093CE008091C80086FFFCCF8B
:10E670008091C80080648093C8003196992379F70F
:10E680000895282F982F92959F70892F805D8A3347
:10E6900008F0895F8093CE008091C80086FFFCCF90
:10E6A0008091C80080648093C800822F8F70982F5B
:10E6B000905D9A3308F0995F9093CE008091C800E6
:10E6C00086FFFCCF8091C80080648093C8000895C5
:10E6D0009C01FB01853691051CF46330710594F0B3
:10E6E000C90164E670E00F94BEFE605D7F4F6093E9
:10E6F000CE008091C80086FFFCCF8091C800806466
:10E700008093C8002B30310514F43297B4F0C9015E
:10E7100064E670E00F94BEFE6AE070E00F94BEFE07
:10E72000605D7F4F6093CE008091C80086FFFCCF74
:10E730008091C80080648093C800C9016AE070E0DD
:10E740000F94BEFEC0968093CE008091C80086FFD5
:10E75000FCCF8091C80080648093C80008958770C2
:10E76000806480937C0080917A00806480937A003A
:10E7700080917A0086FDFCCF20917800409179004D
:10E78000942F80E030E0282B392BC90108951F9386
:10E79000182F88E692EE60E00F94F2F21093CE000C
:10E7A0008091C80086FFFCCF8091C8008064809370
:10E7B000C8000F9410F31F9108952F923F924F922B
:10E7C0005F926F927F928F929F92AF92BF92CF9201
:10E7D000DF92EF92FF920F931F93DF93CF93CDB70A
:10E7E000DEB762970FB6F894DEBF0FBECDBF382EEE
:10E7F000622ECA01DB015C016D01772420E2222E2A
:10E800002E010894411C511C8BC081E0A81680E0A9
:10E81000B80681E0C80680E0D80628F0C601AA271D
:10E82000BB270F9441F3BB27AD2D9C2D8B2D0F944F
:10E8300041F38A2D0F9441F32092CE008091C800BD
:10E8400086FFFCCF8091C80080648093C8009DE261
:10E850009093CE008091C80086FFFCCF8091C800C5
:10E8600080648093C8002092CE008091C80086FF0B
:10E87000FCCF8091C80080648093C8001982860113
:10E88000750188249924A1E03A1651F03A1620F037
:10E89000B2E03B1661F409C00BBFF701779007C0E7
:10E8A000C7010F94E5FE782E02C0F7017080872D16
:10E8B0000F9441F32092CE008091C80086FFFCCFD8
:10E8C0008091C80080648093C800872D8052F40135
:10E8D000EF70F0708F3520F4E40DF51D708204C0E8
:10E8E000E40DF51D8EE280830894E11CF11C011DEE
:10E8F000111D0894811C911C90E18916910409F066
:10E90000C2CF80E190E0A0E0B0E0A80EB91ECA1E20
:10E91000DB1E198AC2010F942EF30F9410F36A9430
:10E92000662009F072CF62960FB6F894DEBF0FBE74
:10E93000CDBFCF91DF911F910F91FF90EF90DF90AE
:10E94000CF90BF90AF909F908F907F906F905F908F
:10E950004F903F902F9008952F923F924F925F9249
:10E960006F927F928F929F92AF92BF92CF92DF92DF
:10E97000EF92FF920F931F93DF93CF93CDB7DEB744
:10E98000CD53D1400FB6F894DEBF0FBECDBF80ECA3
:10E9900081B98CE782B980E090E020ED37E0F901A1
:10E9A0003197F1F701968A3F9105C9F780B18C73D1
:10E9B000883171F080E090E0A0E0B0E0ABBFFC01F6
:10E9C000879196918F5F9F4F19F0EE27FF2709944B
:10E9D0009FEF97B987E384B980EC85B988E08AB95D
:10E9E0009BB982E08DB99EB98091C8008260809306
:10E9F000C80082E28093CC0088E18093C9000000C7
:10EA000020E030E040E050E0E0E4F1E060E070E081
:10EA100011C0CF010197F1F72F5F3F4F4F4F5F4F6D
:10EA2000213E17E6310715E3410710E0510710F0CA
:10EA300061E070E08091C80087FD03C06115710539
:10EA400041F39B012F5F3F4FC25EDE4F3983288326
:10EA5000CE51D140C25EDE4F48815981CE51D14066
:10EA60004130510511F00D94ADFEC05DDE4F1982AD
:10EA70001882C053D14060E0C15DDE4F1882CF5292
:10EA8000D140AA24BB24C05EDE4F188219821A82AC
:10EA90001B82C052D140CE5CDE4F188219821A828E
:10EAA0001B82C253D14080E090E0A0E0B0E0ABBF59
:10EAB000FC01A791B691C45CDE4FB983A883CC5307
:10EAC000D1400D94A8FEC25EDE4FE881F981CE519F
:10EAD000D140319709F52091CE00C25EDE4F1982F8
:10EAE0001882CE51D14022C02F5F3F4F4F4F5F4F12
:10EAF0002130F2E13F07FAE74F07F0E05F0780F0CF
:10EB0000C45CDE4F08811981CC53D1400F5F1F4F89
:10EB100019F0EE27FF27099420E030E040E050E0B4
:10EB20008091C80087FFE0CF2091CE00213209F00C
:10EB30000DC60894A11CB11C33E0A316B10409F062
:10EB400007C600E010E018C041E24093CE0080917B
:10EB5000C80086FFFCCF8091C80080648093C80005
:10EB60002F5F3F4F2931310579F70F9410F30F5F75
:10EB70001F4F0530110519F020E030E0E5CF10926D
:10EB800008021092090210920A0210920B021092CF
:10EB900004021092050210920602109207021092CF
:10EBA000000210920102109202021092030287EDFD
:10EBB00090EE60E00F9429F388EF90EE60E00F9400
:10EBC000F2F28091C80087FFFCCF9091CE00903682
:10EBD00008F09F759032B8F09093CE008091C800F5
:10EBE00086FFFCCF8091C80080648093C80080E2DB
:10EBF0008093CE008091C80086FFFCCF8091C80032
:10EC000080648093C800983409F4DBC19934B8F467
:10EC1000923409F45DC1933458F4903319F1903370
:10EC200008F491C59F33A1F1903409F08CC5BDC0A3
:10EC3000953409F474C1963409F085C59CC19235A8
:10EC400009F423C2933538F49C3409F4F9C19135A1
:10EC500009F079C510C2963509F43DC2993509F01D
:10EC600072C590C48DE692EE62E00F9429F3109283
:10EC700004021092050210920602109207021092EE
:10EC800008021092090210920A0210920B0217C198
:10EC900081E892EE62E00F9429F387ED90EE60E058
:10ECA0000F9429F389E091EE60E00F94F2F289EA83
:10ECB00091EE60E00F9429F389E191EE60E00F940A
:10ECC000F2F28CEC90EE60E00F9429F389E291EE81
:10ECD00060E00F94F2F286E090E061E070E00F9463
:10ECE00068F30F9410F389E491EE60E00F94F2F270
:10ECF0008BEB91EE60E00F9429F389E391EE60E0F5
:10ED00000F94F2F285EB91EE60E00F9429F389E520
:10ED100091EE60E00F94F2F28EE10F9441F388E9F6
:10ED20000F9441F382E00F9441F30F9410F389E6BE
:10ED300091EE60E00F94F2F219E0E0E0F0E0109361
:10ED40005700E4918E2F0F9441F30F9410F389E74D
:10ED500091EE60E00F94F2F2E3E0F0E010935700E0
:10ED6000E4918E2F0F9441F30F9410F389E891EE04
:10ED700060E00F94F2F2E2E0F0E010935700E491CB
:10ED80008E2F0F9441F30F9410F389E991EE60E018
:10ED90000F94F2F2E1E0F0E0109357001491812F0C
:10EDA0000F9441F30F9410F307CF8DE892EE62E0D9
:10EDB0000F9429F38DE392EE60E00F9429F30F9402
:10EDC00010F300E010E019C0C8016F2D0F94EDFEA4
:10EDD000FF2031F48BE392EE60E00F94F2F20BC06F
:10EDE000F092CE008091C80086FFFCCF8091C800D1
:10EDF00080648093C8000F5F1F4FC80189529F41F4
:10EE0000AA2797FDA095BA2FABBFFC01F7905AE255
:10EE1000F51621F062E000301607B1F60F9410F3FA
:10EE20000F9410F389E492EE60E00F9429F30F94AD
:10EE300010F3CC24DD2400E010E01EC0C8010F94C4
:10EE4000E5FEF82E882331F48BE392EE60E00F9418
:10EE5000F2F20BC08093CE008091C80086FFFCCFF9
:10EE60008091C80080648093C800FE1419F0089453
:10EE7000C11CD11C0F5F1F4FC80189529F41AA2797
:10EE800097FDA095BA2FABBFFC01E7907AE2E71699
:10EE900021F082E00030180789F60F9410F30F94E8
:10EEA00010F384E592EE60E00F94F2F2C60161E0A7
:10EEB00070E00F9468F30F9410F30F9410F3109216
:10EEC000000210920102109202021092030274CE0C
:10EED0008BE992EE62E00F9429F30B9A139A16C015
:10EEE000139880E090E0E0EDF7E03197F1F70196BC
:10EEF00084369105C1F7139A80E090E0E0EDF7E0E9
:10EF00003197F1F7019684369105C1F78091C800D9
:10EF100087FFE6CF8091C80087FFFCCF0EC487EA49
:10EF200092EE62E00F9429F34091000250910102A9
:10EF3000609102027091030281E020E10F94DDF301
:10EF40008091000290910102A0910202B09103020F
:10EF500080509F4FAF4FBF4F8093000290930102AC
:10EF6000A0930202B093030280509041A040B040B1
:10EF700008F422CEA4CF85EB92EE62E00F9429F341
:10EF800040910402509105026091060270910702BF
:10EF900080E020E10F94DDF380910402909105025E
:10EFA000A0910602B091070280509F4FAF4FBF4F14
:10EFB0008093040290930502A0930602B093070287
:10EFC000FBCD82EC92EE62E00F9429F38DE692EE97
:10EFD00060E00F9429F381E892EE60E00F9429F34A
:10EFE0008DE892EE60E00F9429F38BE992EE60E0F9
:10EFF0000F9429F387EA92EE60E00F9429F385EBF2
:10F0000092EE60E00F9429F382EC92EE60E00F94B0
:10F0100029F389EC92EE60E00F9429F38AED92EEE9
:10F0200060E00F9429F384EF92EE60E00F9429F3EF
:10F030008FEF92EE60E00F9429F388E193EEB9CD63
:10F0400089EC92EE62E00F9429F381E40F94C7F308
:10F0500082E40F94C7F383E40F94C7F384E40F941E
:10F06000C7F385E40F94C7F386E40F94C7F387E4EE
:10F070000F94C7F3A1CD8AED92EE62E00F9429F3CD
:10F0800099249394AA24BB24CAC384EF92EE62E02D
:10F090000F9429F3409108025091090260910A02ED
:10F0A00070910B0282E020E10F94DDF38091080261
:10F0B00090910902A0910A02B0910B0280509F4FDB
:10F0C000AF4FBF4F8093080290930902A0930A02AA
:10F0D000B0930B0271CD8FEF92EE62E00F9429F3A3
:10F0E0008CEC90EE60E00F9429F381EC91EE60E0FF
:10F0F0000F9429F30BE015EECC5DDE4F19830883E6
:10F10000C452D140662477244301CA5DDE4F198280
:10F110001882C652D140A401930156954795379560
:10F120002795C85DDE4F288339834A835B83C852A5
:10F13000D140CA5DDE4F48815981C652D1404F5FF0
:10F140005F4FCA5DDE4F59834883C652D140CA0122
:10F1500062E070E00F9468F350E25093CE0080912B
:10F16000C80086FFFCCF8091C80080648093C800EF
:10F170006DE26093CE008091C80086FFFCCF809145
:10F18000C80080648093C80070E27093CE008091C4
:10F19000C80086FFFCCF8091C80080648093C800BF
:10F1A000C85DDE4FE880F9800A811B81C852D140DA
:10F1B000BB27A12F902F8F2D0F9441F3C85DDE4FF9
:10F1C0008881C852D1400F9441F370E2F72EF0923B
:10F1D000CE008091C80086FFFCCF8091C80080647B
:10F1E0008093C8000DE30093CE008091C80086FF95
:10F1F000FCCF8091C80080648093C80010E2109317
:10F20000CE008091C80086FFFCCF8091C80080644A
:10F210008093C8008BBEF3012791C45DDE4F288325
:10F22000CC52D140A22EBB24CC24DD240894611CF6
:10F23000711C811C911C8BBEF3018791282E3324F5
:10F2400044245524142D032DF22CEE24EA0CFB1C2F
:10F250000C1D1D1D0894611C711C811C911C8BBE12
:10F26000F3013791C35DDE4F3883CD52D14008940E
:10F27000611C711C811C911C8BBEF3014791C25D06
:10F28000DE4F4883CE52D1402DEF3FEF4FEF5FEF7F
:10F29000620E731E841E951E0F9441F330E230936C
:10F2A000CE008091C80086FFFCCF8091C8008064AA
:10F2B0008093C800C45DDE4F8881CC52D1400F944A
:10F2C00041F340E24093CE008091C80086FFFCCF1E
:10F2D0008091C80080648093C800C25DDE4F888141
:10F2E000CE52D1400F9441F350E25093CE00809122
:10F2F000C80086FFFCCF8091C80080648093C8005E
:10F30000C35DDE4F8881CD52D1400F9441F360E25E
:10F310006093CE008091C80086FFFCCF8091C8002A
:10F3200080648093C8007FEFE7167FEFF70670E0F8
:10F33000070770E0170731F486EF91EE60E00F9455
:10F34000F2F2DFC0D801C7018070907CA070B0706D
:10F350008050904CA040B040D1F52FEF3FE340E00B
:10F3600050E0E222F32204231523C85DDE4FA8807B
:10F37000B980CA80DB80C852D140AE0CBF1CC01E11
:10F38000D11EAA0CBB1CCC1CDD1C80E092EE60E000
:10F390000F94F2F2BB27A12F902F8F2D0F9441F3E2
:10F3A0008E2D0F9441F330E23093CE008091C8004F
:10F3B00086FFFCCF8091C80080648093C8004EE334
:10F3C0004093CE008091C80086FFFCCF87C06EE0DE
:10F3D0007EEF80E090E0E622F722082319237CE00C
:10F3E000E71674E9F70670E0070770E0170709F001
:10F3F00088C0C25DDE4F8881CE52D140E82EFF2406
:10F4000000E010E0102F0F2DFE2CEE24C35DDE4F28
:10F410009881CD52D140E90EF11C011D111DD6017C
:10F42000C50181709070A070B070DC0199278827A9
:10F43000E80EF91E0A1F1B1F20EF30E040E050E0ED
:10F44000A222B322C422D522F1E1AA0CBB1CCC1CFF
:10F45000DD1CFA95D1F7EA0CFB1C0C1D1D1D41E0CB
:10F4600050E060E070E02422352246225722E5E198
:10F47000220C331C441C551CEA95D1F7E20CF31CFA
:10F48000041D151D57016801AA0CBB1CCC1CDD1CFA
:10F4900087E092EE60E00F94F2F2C801AA27BB2742
:10F4A0000F9441F3BB27A12F902F8F2D0F9441F381
:10F4B0008E2D0F9441F350E25093CE008091C800FE
:10F4C00086FFFCCF8091C80080648093C8006EE303
:10F4D0006093CE008091C80086FFFCCF8091C80069
:10F4E00080648093C800C601AA27BB270F9441F30C
:10F4F000BB27AD2D9C2D8B2D0F9441F38A2D0F949E
:10F5000041F370E27093CE008091C80086FFFCCF7B
:10F510008091C80080648093C800CC5DDE4FE88194
:10F52000F981C452D140CF01AA2797FDA095BA2FE7
:10F53000ABBFFC018791969160E00F94F2F20F94BB
:10F5400010F3CC5DDE4F08811981C452D1400E5FAB
:10F550001F4FCC5DDE4F19830883C452D140CA5D72
:10F56000DE4F28813981C652D1402333310509F459
:10F5700023CB44E050E060E070E0640E751E861E10
:10F58000971EC9CD88E193EE62E00F9429F38CE0D9
:10F5900092EE60E00F94F2F28091C80087FFFCCFFA
:10F5A0001091CE001F751093CE008091C80086FF89
:10F5B000FCCF8091C80080648093C8000F9410F342
:10F5C000812F81548A3108F0BBC0143409F456C02D
:10F5D000153440F4123431F11334D0F5113409F0FC
:10F5E000A5C00AC0163409F475C0163408F45CC00E
:10F5F000173409F09BC084C08FEF81B90DC082B170
:10F60000809582B980E090E0E0EDF7E03197F1F786
:10F610000196883C9105C1F78091C80087FFEFCF24
:10F6200012B887C08FEF84B90DC085B1809585B9B8
:10F6300080E090E0E0EDF7E03197F1F70196883C4B
:10F640009105C1F78091C80087FFEFCF15B871C051
:10F650008FEF87B90DC088B1809588B980E090E0C0
:10F66000E0EDF7E03197F1F70196883C9105C1F79D
:10F670008091C80087FFEFCF18B85BC08FEF8AB9C1
:10F680000DC08BB180958BB980E090E0E0EDF7E0A4
:10F690003197F1F70196883C9105C1F78091C80038
:10F6A00087FFEFCF1BB845C08FEF8DB90DC08EB16E
:10F6B00080958EB980E090E0E0EDF7E03197F1F7CA
:10F6C0000196883C9105C1F78091C80087FFEFCF74
:10F6D0001EB82FC08FEF80BB0DC081B3809581BB5A
:10F6E00080E090E0E0EDF7E03197F1F70196883C9B
:10F6F0009105C1F78091C80087FFEFCF11BA19C0FB
:10F700008FEF83BB0DC084B3809584BB80E090E015
:10F71000E0EDF7E03197F1F70196883C9105C1F7EC
:10F720008091C80087FFEFCF14BA03C087E192EE43
:10F7300040CA8091C80087FFFCCF8091CE003CCAB0
:10F740008AE292EE36CA84E091EE33CAAA24BB2440
:10F75000933061F1943028F4913089F0923008F5BB
:10F7600008C09530B1F1953040F1963009F053C0A2
:10F770004EC02B3109F0A7C991E06BE1A4C921303B
:10F7800041F0C15DDE4F5881CF52D140251709F0BD
:10F79000F2C26227C15DDE4F2883CF52D14092E092
:10F7A00092C9B22FA0E0622793E08DC9822F90E02A
:10F7B000A82BB92B622794E086C92E3009F0DBC252
:10F7C000622795E0C05DDE4F19821882C053D14098
:10F7D0007AC9E1E0F0E0EC0FFD1FC05DDE4FE8808C
:10F7E000F980C053D140EE0DFF1D208387010F5FCC
:10F7F0001F4FC05DDE4F19830883C053D14062277D
:10F800000A171B0709F05FC9D80196E05CC92617E3
:10F8100009F0B1C203C0973009F055C99924898114
:10F82000833109F4FCC08431C8F4863009F4C2C0C5
:10F83000873050F4823009F4F0C0833009F458C0A6
:10F84000813009F00AC23EC0813109F462C08231C0
:10F8500008F0A6C0803109F000C2DFC0883109F489
:10F8600072C0893150F4853109F4D9C0853108F46A
:10F8700077C1863109F0F1C173C18A3109F457C0EB
:10F880008A3108F47CC08B3109F446C08D3109F00F
:10F89000E4C18D81803311F090E00AC08F8188230C
:10F8A00011F49EE105C0813011F092E001C098E9A9
:10F8B0001A821B828D818C831D829E831F8227E08A
:10F8C00030E0CFC11A8288E08B8381E48C8386E5A7
:10F8D0008D8382E58E8389E48F8383E5888780E545
:10F8E00089878FE58A8782E38B872BE030E0B9C177
:10F8F0008A81813941F0823941F0803911F48FE0F9
:10F9000005C080E003C082E001C08AE01A828B83D8
:10F9100044C09924939481C08D81882311F48EE191
:10F920002CC0813011F082E028C088E926C01A82FC
:10F93000E1E0F0E089E08093570084918B831C82A2
:10F9400024E030E08EC18B81803589F48C81883051
:10F9500039F4E2E0F0E089E08093570084910DC033
:10F96000E0E0F0E089E080935700849106C0E3E096
:10F97000F0E089E08093570084911A82DFCF8D8177
:10F98000836C99E0E1E0F0E0082E90935700E89551
:10F9900007B600FCFDCF1A821B8223E030E061C174
:10F9A0001A82CE5CDE4F188219821A821B82C253E1
:10F9B000D14055C18A8190E0A0E0B0E0582F4427A3
:10F9C000332722278B8190E0A0E0B0E0DC0199276B
:10F9D0008827282B392B4A2B5B2B8D8190E0A0E0C8
:10F9E000B0E0282B392B4A2B5B2B8C8190E0A0E0D8
:10F9F000B0E0BA2FA92F982F8827282B392B4A2B14
:10FA00005B2B220F331F441F551FC05EDE4F288320
:10FA100039834A835B83C052D1401A8220C19A81C4
:10FA20002B81833149F0C05EDE4F488159816A8164
:10FA30007B81C052D1408AC0CE5CDE4F4881598163
:10FA40006A817B81C253D140403080EC580783E00B
:10FA5000680780E07807F0F483E0FA0160935B00C8
:10FA600080935700E89507B600FCFDCFCE5CDE4FD3
:10FA7000488159816A817B81C253D14040505F4F98
:10FA80006F4F7F4FCE5CDE4F488359836A837B8301
:10FA9000C253D140C95CDE4F9883C753D140CA5C82
:10FAA000DE4F1882C653D140022F10E0CA5CDE4FF1
:10FAB00068817981C653D140062B172BC05EDE4F7B
:10FAC000488159816A817B81C052D140DE011B96F9
:10FAD00031E08C9111962C9111971296C75CDE4FF4
:10FAE0002883C953D140C85CDE4F1882C853D14027
:10FAF00090E0C85CDE4FE881F981C853D1408E2B7D
:10FB00009F2B0C01FA0160935B0030935700E8953E
:10FB100011244E5F5F4F6F4F7F4F02501040C9F668
:10FB200085E0C05EDE4FE880F9800A811B81C0520B
:10FB3000D140F70100935B0080935700E89507B62A
:10FB400000FCFDCF81E180935700E8951A82C05EEA
:10FB5000DE4F488359836A837B83C052D1407FC084
:10FB6000FA80C55CDE4FF882CB53D140C65CDE4FD5
:10FB70001882CA53D1408B81C82EDD24C65CDE4F6B
:10FB800008811981CA53D140C02AD12A1A82898199
:10FB9000BE016D5F7F4F843121F59601C05EDE4F5F
:10FBA000E880F9800A811B81C052D1400BBFF70168
:10FBB00087919691DB018C9311969C936E5F7F4F9A
:10FBC000D801C7010296A11DB11DC05EDE4F88831A
:10FBD0009983AA83BB83C052D14022503040F1F6B2
:10FBE00036C0C05EDE4F288139814A815B81C052B8
:10FBF000D1400894C108D108760100E010E00894D3
:10FC0000C11CD11C0894E11CF11C011D111DE20E48
:10FC1000F31E041F151F21BDBB27A52F942F832F73
:10FC200082BD2F5F3F4F4F4F5F4FF89A80B5DB018A
:10FC30008D93BD012E153F054007510761F7C05E4A
:10FC4000DE4F288339834A835B83C052D1409601BB
:10FC50002D5F3F4FFB01108204C080EC8A8322E0BD
:10FC600030E08BE18093CE008091C80086FFFCCF0E
:10FC70008091C80080648093C800C15DDE4FF88128
:10FC8000CF52D140F093CE008091C80086FFFCCFC8
:10FC90008091C80080648093C800432F3093CE00C9
:10FCA0008091C80086FFFCCF8091C800806480935B
:10FCB000C800922F2093CE008091C80086FFFCCF11
:10FCC0008091C80080648093C8008EE08093CE004D
:10FCD0008091C80086FFFCCF8091C800806480932B
:10FCE000C80065E1C15DDE4FE880CF52D1406E258E
:10FCF00069276427FE01319610C090819093CE0051
:10FD00008091C80086FFFCCF31968091C800806446
:10FD10008093C8006927215030402115310569F7CB
:10FD20006093CE008091C80086FFFCCF8091C80010
:10FD300080648093C800992081F4C15DDE4F088102
:10FD4000CF52D1400F5FC15DDE4F0883CF52D1400B
:10FD500090E0A0E0B0E00D9463F500008091C80051
:10FD60008D7F8093C80081E180935700E895EE274E
:10FD7000FF270994FFCF90E00D9463F597FB092EC0
:10FD800007260AD077FD04D00CD006D000201AF444
:10FD9000709561957F4F0895F6F7909581959F4FE7
:10FDA0000895AA1BBB1B51E107C0AA1FBB1FA617C2
:10FDB000B70710F0A61BB70B881F991F5A95A9F714
:10FDC00080959095BC01CD010895F999FECF92BD23
:10FDD00081BDF89A992780B50895262FF999FECF0D
:10FDE0001FBA92BD81BD20BD0FB6F894FA9AF99A58
:0AFDF0000FBE01960895F894FFCFAE
:040000033000E000E9
:00000001FF
